:020000040000FA
:04000000A0EFBFF0BE
:020000040001F9
:087F3800000000000000000041
:107F4000240EAC6E200EAF6E900EAB6E46D8C108FC
:107F500053E1570EAD6E4B0EAD6E006A3ED8F86E13
:107F6000076E3BD8F76EA96E38D8F66EA86E35D876
:107F7000016E012A00EE09F0F56E2FD8EC6E012E8D
:107F8000FBD700661FD007AC03D0040E1ED818D054
:107F900007AE04D00C00C40E18D812D0940E15D819
:107FA0000A00080E056E00EE0AF0080E066EEE508E
:107FB000F56E0F00062EFBD7840E07D8052EF5D7D9
:107FC000A694C9D74E0EAD6EC8D7A66E550EA76E35
:107FD000AA0EA76EA682000012000B0E026E036AA4
:107FE000046A9EAA03D0AE5000261200042EF9D7D0
:0C7FF000032EF6D7022EF3D7AB9E9ED7CF
:020000040030CA
:0E000000FF32F8E0FFFD8AFFFFFFFFFFFF0069
:0200000400F00A
:10000000426F6F746C6F61642E2031304D687A00DE
:100010007061756C666A756A6F2E667265652E0012
:100020004D50414C41422076382E3932202020005C
:100030002031392F30332F3230313620202020002C
:00000001FF
